
 Start         Length     Name                   Class
 0001:00401000 0000017A5H _TEXT                  CODE
 0002:00403000 000001914H _DATA                  DATA
 0003:00404914 0000000A4H _BSS                   BSS
 0004:00000000 00000009CH _TLS                   TLS


Detailed map of segments
 0001:00000000 00000236 C=CODE    S=_TEXT    G=(none)   M=C:\PROGRAM FILES\BORLAND\BCC55\LIB\C0D32.OBJ ACBP=A9
 0001:00000238 00000555 C=CODE    S=_TEXT    G=(none)   M=C:\PROGRAMS\IBM\SOM\SAMPLES\SOMD\CPP\EVENT\EVENTCOM.OBJ ACBP=A9
 0001:00000790 00000AEC C=CODE    S=_TEXT    G=(none)   M=C:\PROGRAMS\IBM\SOM\SAMPLES\SOMD\CPP\EVENT\EVENTCH.OBJ ACBP=A9
 0001:0000127C 000001E1 C=CODE    S=_TEXT    G=(none)   M=C:\PROGRAMS\IBM\SOM\SAMPLES\SOMD\CPP\EVENT\CELL.OBJ ACBP=A9
 0001:00001460 000000B4 C=CODE    S=_TEXT    G=(none)   M=C:\PROGRAMS\IBM\SOM\SAMPLES\SOMD\CPP\EVENT\EVENTI.OBJ ACBP=A9
 0001:00001514 00000001 C=CODE    S=_TEXT    G=(none)   M=C:\PROGRAM FILES\BORLAND\BCC55\LIB\CW32MTI.LIB|crtlst_i ACBP=A9
 0001:00001518 00000001 C=CODE    S=_TEXT    G=(none)   M=C:\PROGRAM FILES\BORLAND\BCC55\LIB\CW32MTI.LIB|crtlst_e ACBP=A9
 0001:0000151C 00000001 C=CODE    S=_TEXT    G=(none)   M=C:\PROGRAM FILES\BORLAND\BCC55\LIB\CW32MTI.LIB|crtlst_l ACBP=A9
 0001:00001520 0000009F C=CODE    S=_TEXT    G=(none)   M=C:\PROGRAM FILES\BORLAND\BCC55\LIB\CW32MTI.LIB|xxv ACBP=A9
 0001:000015C0 00000070 C=CODE    S=_TEXT    G=(none)   M=C:\PROGRAM FILES\BORLAND\BCC55\LIB\CW32MTI.LIB|xxa ACBP=A9
 0001:00001630 00000018 C=CODE    S=_TEXT    G=(none)   M=C:\PROGRAM FILES\BORLAND\BCC55\LIB\CW32MTI.LIB|libmain ACBP=A9
 0001:00001648 0000003C C=CODE    S=_TEXT    G=(none)   M=C:\PROGRAM FILES\BORLAND\BCC55\LIB\CW32MTI.LIB|dlllock ACBP=A9
 0002:0000000C 00000104 C=DATA    S=_DATA    G=DGROUP   M=C:\PROGRAM FILES\BORLAND\BCC55\LIB\C0D32.OBJ ACBP=A9
 0002:00000110 000008F4 C=DATA    S=_DATA    G=DGROUP   M=C:\PROGRAMS\IBM\SOM\SAMPLES\SOMD\CPP\EVENT\EVENTCOM.OBJ ACBP=A9
 0002:00000A04 00000A40 C=DATA    S=_DATA    G=DGROUP   M=C:\PROGRAMS\IBM\SOM\SAMPLES\SOMD\CPP\EVENT\EVENTCH.OBJ ACBP=A9
 0002:00001444 000003A0 C=DATA    S=_DATA    G=DGROUP   M=C:\PROGRAMS\IBM\SOM\SAMPLES\SOMD\CPP\EVENT\CELL.OBJ ACBP=A9
 0002:000017E4 0000002C C=DATA    S=_DATA    G=DGROUP   M=C:\PROGRAMS\IBM\SOM\SAMPLES\SOMD\CPP\EVENT\EVENTI.OBJ ACBP=A9
 0002:00001810 000000C4 C=DATA    S=_DATA    G=DGROUP   M=C:\PROGRAM FILES\BORLAND\BCC55\LIB\CW32MTI.LIB|xxv ACBP=A9
 0002:000018C0 00000004 C=DATA    S=_DATA    G=DGROUP   M=C:\PROGRAM FILES\BORLAND\BCC55\LIB\CW32MTI.LIB|xx_w ACBP=A9
 0002:000018C4 00000004 C=DATA    S=_DATA    G=DGROUP   M=C:\PROGRAM FILES\BORLAND\BCC55\LIB\CW32MTI.LIB|cfinfo ACBP=A9
 0002:000018C8 00000004 C=DATA    S=_DATA    G=DGROUP   M=C:\PROGRAM FILES\BORLAND\BCC55\LIB\CW32MTI.LIB|xinitcvt ACBP=A9
 0002:000018CC 00000004 C=DATA    S=_DATA    G=DGROUP   M=C:\PROGRAM FILES\BORLAND\BCC55\LIB\CW32MTI.LIB|wildptr ACBP=A9
 0002:000018D0 00000004 C=DATA    S=_DATA    G=DGROUP   M=C:\PROGRAM FILES\BORLAND\BCC55\LIB\CW32MTI.LIB|wwildptr ACBP=A9
 0002:000018D4 00000028 C=DATA    S=_DATA    G=DGROUP   M=C:\PROGRAM FILES\BORLAND\BCC55\LIB\CW32MTI.LIB|dlllock ACBP=A9
 0002:000018FC 00000018 C=DATA    S=_DATA    G=DGROUP   M=<internal> ACBP=A9
 0003:00000000 00000044 C=BSS     S=_BSS     G=DGROUP   M=C:\PROGRAMS\IBM\SOM\SAMPLES\SOMD\CPP\EVENT\EVENTCOM.OBJ ACBP=A9
 0003:00000044 00000034 C=BSS     S=_BSS     G=DGROUP   M=C:\PROGRAMS\IBM\SOM\SAMPLES\SOMD\CPP\EVENT\EVENTCH.OBJ ACBP=A9
 0003:00000078 0000001C C=BSS     S=_BSS     G=DGROUP   M=C:\PROGRAMS\IBM\SOM\SAMPLES\SOMD\CPP\EVENT\CELL.OBJ ACBP=A9
 0003:00000094 00000008 C=BSS     S=_BSS     G=DGROUP   M=C:\PROGRAM FILES\BORLAND\BCC55\LIB\CW32MTI.LIB|xxv ACBP=A9
 0003:0000009C 00000004 C=BSS     S=_BSS     G=DGROUP   M=C:\PROGRAM FILES\BORLAND\BCC55\LIB\CW32MTI.LIB|rawdll ACBP=A9
 0003:000000A0 00000004 C=BSS     S=_BSS     G=DGROUP   M=C:\PROGRAM FILES\BORLAND\BCC55\LIB\CW32MTI.LIB|dlllock ACBP=A9
 0004:00000000 0000009C C=TLS     S=_TLS     G=DGROUP   M=C:\PROGRAM FILES\BORLAND\BCC55\LIB\CW32MTI.LIB|xxv ACBP=A9

  Address         Publics by Name

 0001:00001434      Cell::_get_val(Environment *)
 0001:00001420      Cell::notifyEventCh(Environment *)
 0001:000013BC      CellNewClass
 0001:00001630      DllEntryPoint
 0001:000014CF      DllMain
 0001:00000E7C      EventChannelAdmin_ConsumerAdmin::EventChannelAdmin_ConsumerAdmin()
 0001:00001220      EventChannelAdmin_ConsumerAdmin::operator delete(void *)
 0001:00000E54      EventChannelAdmin_ConsumerAdmin::operator new(unsigned int)
 0001:00000FB8      EventChannelAdmin_ConsumerAdmin::somFree()
 0001:00000B38      EventChannelAdmin_ConsumerAdminNewClass
 0001:00000FCC      EventChannelAdmin_EventChannel::somFree()
 0001:00000C00      EventChannelAdmin_EventChannelNewClass
 0001:00000F24      EventChannelAdmin_SupplierAdmin::EventChannelAdmin_SupplierAdmin()
 0001:00001238      EventChannelAdmin_SupplierAdmin::operator delete(void *)
 0001:00000EFC      EventChannelAdmin_SupplierAdmin::operator new(unsigned int)
 0001:00000FA4      EventChannelAdmin_SupplierAdmin::somFree()
 0001:00000B9C      EventChannelAdmin_SupplierAdminNewClass
 0001:00000DDC      EventComm_Consumer::EventComm_Consumer()
 0001:00000724      EventComm_Consumer::_get_ev_con(Environment *)
 0001:0000074C      EventComm_Consumer::_set_ev_con(Environment *, EventComm_EventConnection *)
 0001:00001208      EventComm_Consumer::operator delete(void *)
 0001:00000DB0      EventComm_Consumer::operator new(unsigned int)
 0001:00001448      EventComm_Consumer::push(Environment *, any *)
 0001:00000650      EventComm_ConsumerNewClass
 0001:00000C90      EventComm_EventConnection::EventComm_EventConnection()
 0001:00000738      EventComm_EventConnection::disconnect(Environment *)
 0001:000011A4      EventComm_EventConnection::operator delete(void *)
 0001:00000C64      EventComm_EventConnection::operator new(unsigned int)
 0001:00000710      EventComm_EventConnection::somFree()
 0001:000005D4      EventComm_EventConnectionNewClass
 0001:00000D38      EventComm_Supplier::EventComm_Supplier()
 0001:00000764      EventComm_Supplier::_get_ev_con(Environment *)
 0001:00000778      EventComm_Supplier::_set_ev_con(Environment *, EventComm_EventConnection *)
 0001:000011F0      EventComm_Supplier::operator delete(void *)
 0001:00000D0C      EventComm_Supplier::operator new(unsigned int)
 0001:000006B0      EventComm_SupplierNewClass
 0001:00000638      SOMClass::somCheckVersion(long, long)
 0001:000014C1      SOMInitModule
 0001:00000FE0      SOMObject::SOMObject()
 0001:00001264      SOMObject::operator delete(void *)
 0001:00001008      SOMObject::somDefaultInit(somInitCtrlStruct *)
 0001:00001250      SOMObject::somFree()
 0001:00000202      Sysinit::__linkproc__ __fastcall GetTls()
 0002:0000145C      _CellCClassData
 0002:00001448      _CellClassData
 0002:00000A14      _EventChannelAdmin_ConsumerAdminCClassData
 0002:00000A08      _EventChannelAdmin_ConsumerAdminClassData
 0002:00000E60      _EventChannelAdmin_EventChannelCClassData
 0002:00000E50      _EventChannelAdmin_EventChannelClassData
 0002:00000C38      _EventChannelAdmin_SupplierAdminCClassData
 0002:00000C2C      _EventChannelAdmin_SupplierAdminClassData
 0002:00000300      _EventComm_ConsumerCClassData
 0002:000002F0      _EventComm_ConsumerClassData
 0002:000003C4      _EventComm_Consumer_push_mp_tdcs00b579f0
 0002:0000011C      _EventComm_EventConnectionCClassData
 0002:00000114      _EventComm_EventConnectionClassData
 0002:00000174      _EventComm_EventConnection_disconnect_mp_tdcs00b54400
 0002:000005B0      _EventComm_SupplierCClassData
 0002:000005A0      _EventComm_SupplierClassData
 0002:00000678      _EventComm_Supplier_try_pull_mp_tdcs00b58ce0
 0003:00000094      __DestructorCountPtr
 0001:0000154C      __ExceptInit
 0002:000018AC      __ExceptVarsSize
 0001:00001607      __ExceptionHandler
 0001:000015F9      __ExitExceptBlock
 0001:00000117      __GetExceptDLLinfo
 0001:00001598      __GetExceptDLLinfoInternal
 0001:000015C0      __InitExceptBlockLDTC
 0002:00000108      __PackageInfoTable
 0002:0000008B      __TLS_index
 0002:0000008F      __TLS_index4
 0002:00000104      ___CPPdebugHook
 0002:00000104      ___CPPdebugHook_segment
 0002:00001810      ___CPPexceptionList
 0001:00001648      ___CRTL_DLL_Lock
 0001:0000166C      ___CRTL_DLL_Unlock
 0001:0000151C      ___CRTL_VCLLIB_Linkage
 0001:00001518      ___CRTL_VCL_Exit
 0001:00001514      ___CRTL_VCL_Init
 0002:0000182C      ___ExceptStaticXbuff
 0001:00000202      ___System__GetTls
 0002:00001814      ___exceptFlags
 0002:00001828      ___exceptMemAllocVars
 0002:00001824      ___exceptStaticBuffP
 0002:00000089      ___isDLL
 0002:00000050      ___isGUI
 0002:00000088      ___isVCLPackage
 0002:000016EC      ___somC_Cell_ClassInfo
 0002:00001530      ___somC_Cell_newNDMethodsArray
 0003:00000078      ___somC_Cell_parentMtabs
 0002:00000C24      ___somC_EventChannelAdmin_ConsumerAdmin_ClassInfo
 0002:00000AB8      ___somC_EventChannelAdmin_ConsumerAdmin_newNDMethodsArray
 0003:00000044      ___somC_EventChannelAdmin_ConsumerAdmin_parentMtabs
 0002:000010B8      ___somC_EventChannelAdmin_EventChannel_ClassInfo
 0002:00000F24      ___somC_EventChannelAdmin_EventChannel_newNDMethodsArray
 0003:00000064      ___somC_EventChannelAdmin_EventChannel_parentMtabs
 0002:00000E48      ___somC_EventChannelAdmin_SupplierAdmin_ClassInfo
 0002:00000CDC      ___somC_EventChannelAdmin_SupplierAdmin_newNDMethodsArray
 0003:00000054      ___somC_EventChannelAdmin_SupplierAdmin_parentMtabs
 0002:00000598      ___somC_EventComm_Consumer_ClassInfo
 0002:000003F4      ___somC_EventComm_Consumer_newNDMethodsArray
 0003:00000014      ___somC_EventComm_Consumer_parentMtabs
 0002:000002E8      ___somC_EventComm_EventConnection_ClassInfo
 0002:000001A4      ___somC_EventComm_EventConnection_newNDMethodsArray
 0003:00000000      ___somC_EventComm_EventConnection_parentMtabs
 0002:00000850      ___somC_EventComm_Supplier_ClassInfo
 0002:000006AC      ___somC_EventComm_Supplier_newNDMethodsArray
 0003:00000030      ___somC_EventComm_Supplier_parentMtabs
 0002:00001820      ___throwExceptionName
 0002:00001818      ___throwFileName
 0002:0000181C      ___throwLineNumber
 0002:0000008A      ___useDynamicTLS
 0004:00000000      ___xxInfo
 0002:000018C0      ___xxPersonality
 0001:00000000      __acrtused
 0002:000018CC      __argv_expand_ptr
 0002:0000142C      __ectbl__ EventChannelAdmin_ConsumerAdmin::EventChannelAdmin_ConsumerAdmin()
 0002:00001434      __ectbl__ EventChannelAdmin_SupplierAdmin::EventChannelAdmin_SupplierAdmin()
 0002:00001424      __ectbl__ EventComm_Consumer::EventComm_Consumer()
 0002:00001414      __ectbl__ EventComm_EventConnection::EventComm_EventConnection()
 0002:0000141C      __ectbl__ EventComm_Supplier::EventComm_Supplier()
 0002:0000143C      __ectbl__ SOMObject::SOMObject()
 0002:000018C4      __fileinfo
 0001:00000124      __getHInstance
 0002:00000093      __hInstance
 0002:000018FC      __indStub:82
 0002:00001900      __indStub:83
 0002:00001904      __indStub:84
 0002:00001910      __indStub:85
 0002:00001908      __indStub:86
 0002:0000190C      __indStub:87
 0001:0000011C      __isDLL
 0003:0000009C      __pRawDllMain
 0001:00001070      __tpdsc__ EventChannelAdmin_ConsumerAdmin
 0001:00000ECC      __tpdsc__ EventChannelAdmin_ConsumerAdmin *
 0001:0000101C      __tpdsc__ EventChannelAdmin_SupplierAdmin
 0001:00000F74      __tpdsc__ EventChannelAdmin_SupplierAdmin *
 0001:000010C4      __tpdsc__ EventComm_Consumer
 0001:00000E30      __tpdsc__ EventComm_Consumer *
 0001:00001154      __tpdsc__ EventComm_EventConnection
 0001:00000CE4      __tpdsc__ EventComm_EventConnection *
 0001:0000110C      __tpdsc__ EventComm_Supplier
 0001:00000D8C      __tpdsc__ EventComm_Supplier *
 0001:000011BC      __tpdsc__ SOMObject
 0002:000018C8      __turboFloat
 0002:000018D0      __wargv_expand_ptr
 0002:0000085C      _event_data
 0002:00000858      _has_event
 0003:0000009C      b117_0
 0003:000000A0      b119_2
 0003:00000000      b2_2
 0003:00000044      b3_2
 0003:00000078      b4_2
 0003:00000094      b79_2
 0001:00001630      c115_0
 0001:00001648      c119_0
 0001:00000000      c1_0
 0001:00000238      c2_0
 0001:00000790      c3_0
 0001:0000127C      c4_0
 0001:00001460      c5_0
 0001:00001514      c63_0
 0001:00001518      c65_0
 0001:0000151C      c67_0
 0001:00001520      c79_0
 0001:00001520      c79_4
 0001:000015C0      c81_0
 0002:000018CC      d103_0
 0002:000018D0      d105_0
 0002:000018D4      d119_1
 0002:0000000C      d1_1
 0002:00000110      d2_1
 0002:00000A04      d3_1
 0002:00001444      d4_1
 0002:000017E4      d5_1
 0002:00001810      d79_1
 0002:000018C0      d83_0
 0002:000018C4      d87_0
 0002:000018C8      d95_0
 0001:00001484      eventSOMInitTerm
 0004:00000000      t79_3

  Address         Publics by Value

 0001:00000000      __acrtused
 0001:00000000      c1_0
 0001:00000117      __GetExceptDLLinfo
 0001:0000011C      __isDLL
 0001:00000124      __getHInstance
 0001:00000202      ___System__GetTls
 0001:00000202      Sysinit::__linkproc__ __fastcall GetTls()
 0001:00000238      c2_0
 0001:000005D4      EventComm_EventConnectionNewClass
 0001:00000638      SOMClass::somCheckVersion(long, long)
 0001:00000650      EventComm_ConsumerNewClass
 0001:000006B0      EventComm_SupplierNewClass
 0001:00000710      EventComm_EventConnection::somFree()
 0001:00000724      EventComm_Consumer::_get_ev_con(Environment *)
 0001:00000738      EventComm_EventConnection::disconnect(Environment *)
 0001:0000074C      EventComm_Consumer::_set_ev_con(Environment *, EventComm_EventConnection *)
 0001:00000764      EventComm_Supplier::_get_ev_con(Environment *)
 0001:00000778      EventComm_Supplier::_set_ev_con(Environment *, EventComm_EventConnection *)
 0001:00000790      c3_0
 0001:00000B38      EventChannelAdmin_ConsumerAdminNewClass
 0001:00000B9C      EventChannelAdmin_SupplierAdminNewClass
 0001:00000C00      EventChannelAdmin_EventChannelNewClass
 0001:00000C64      EventComm_EventConnection::operator new(unsigned int)
 0001:00000C90      EventComm_EventConnection::EventComm_EventConnection()
 0001:00000CE4      __tpdsc__ EventComm_EventConnection *
 0001:00000D0C      EventComm_Supplier::operator new(unsigned int)
 0001:00000D38      EventComm_Supplier::EventComm_Supplier()
 0001:00000D8C      __tpdsc__ EventComm_Supplier *
 0001:00000DB0      EventComm_Consumer::operator new(unsigned int)
 0001:00000DDC      EventComm_Consumer::EventComm_Consumer()
 0001:00000E30      __tpdsc__ EventComm_Consumer *
 0001:00000E54      EventChannelAdmin_ConsumerAdmin::operator new(unsigned int)
 0001:00000E7C      EventChannelAdmin_ConsumerAdmin::EventChannelAdmin_ConsumerAdmin()
 0001:00000ECC      __tpdsc__ EventChannelAdmin_ConsumerAdmin *
 0001:00000EFC      EventChannelAdmin_SupplierAdmin::operator new(unsigned int)
 0001:00000F24      EventChannelAdmin_SupplierAdmin::EventChannelAdmin_SupplierAdmin()
 0001:00000F74      __tpdsc__ EventChannelAdmin_SupplierAdmin *
 0001:00000FA4      EventChannelAdmin_SupplierAdmin::somFree()
 0001:00000FB8      EventChannelAdmin_ConsumerAdmin::somFree()
 0001:00000FCC      EventChannelAdmin_EventChannel::somFree()
 0001:00000FE0      SOMObject::SOMObject()
 0001:00001008      SOMObject::somDefaultInit(somInitCtrlStruct *)
 0001:0000101C      __tpdsc__ EventChannelAdmin_SupplierAdmin
 0001:00001070      __tpdsc__ EventChannelAdmin_ConsumerAdmin
 0001:000010C4      __tpdsc__ EventComm_Consumer
 0001:0000110C      __tpdsc__ EventComm_Supplier
 0001:00001154      __tpdsc__ EventComm_EventConnection
 0001:000011A4      EventComm_EventConnection::operator delete(void *)
 0001:000011BC      __tpdsc__ SOMObject
 0001:000011F0      EventComm_Supplier::operator delete(void *)
 0001:00001208      EventComm_Consumer::operator delete(void *)
 0001:00001220      EventChannelAdmin_ConsumerAdmin::operator delete(void *)
 0001:00001238      EventChannelAdmin_SupplierAdmin::operator delete(void *)
 0001:00001250      SOMObject::somFree()
 0001:00001264      SOMObject::operator delete(void *)
 0001:0000127C      c4_0
 0001:000013BC      CellNewClass
 0001:00001420      Cell::notifyEventCh(Environment *)
 0001:00001434      Cell::_get_val(Environment *)
 0001:00001448      EventComm_Consumer::push(Environment *, any *)
 0001:00001460      c5_0
 0001:00001484      eventSOMInitTerm
 0001:000014C1      SOMInitModule
 0001:000014CF      DllMain
 0001:00001514      ___CRTL_VCL_Init
 0001:00001514      c63_0
 0001:00001518      c65_0
 0001:00001518      ___CRTL_VCL_Exit
 0001:0000151C      c67_0
 0001:0000151C      ___CRTL_VCLLIB_Linkage
 0001:00001520      c79_4
 0001:00001520      c79_0
 0001:0000154C      __ExceptInit
 0001:00001598      __GetExceptDLLinfoInternal
 0001:000015C0      c81_0
 0001:000015C0      __InitExceptBlockLDTC
 0001:000015F9      __ExitExceptBlock
 0001:00001607      __ExceptionHandler
 0001:00001630      DllEntryPoint
 0001:00001630      c115_0
 0001:00001648      c119_0
 0001:00001648      ___CRTL_DLL_Lock
 0001:0000166C      ___CRTL_DLL_Unlock
 0002:0000000C      d1_1
 0002:00000050      ___isGUI
 0002:00000088      ___isVCLPackage
 0002:00000089      ___isDLL
 0002:0000008A      ___useDynamicTLS
 0002:0000008B      __TLS_index
 0002:0000008F      __TLS_index4
 0002:00000093      __hInstance
 0002:00000104      ___CPPdebugHook
 0002:00000104      ___CPPdebugHook_segment
 0002:00000108      __PackageInfoTable
 0002:00000110      d2_1
 0002:00000114      _EventComm_EventConnectionClassData
 0002:0000011C      _EventComm_EventConnectionCClassData
 0002:00000174      _EventComm_EventConnection_disconnect_mp_tdcs00b54400
 0002:000001A4      ___somC_EventComm_EventConnection_newNDMethodsArray
 0002:000002E8      ___somC_EventComm_EventConnection_ClassInfo
 0002:000002F0      _EventComm_ConsumerClassData
 0002:00000300      _EventComm_ConsumerCClassData
 0002:000003C4      _EventComm_Consumer_push_mp_tdcs00b579f0
 0002:000003F4      ___somC_EventComm_Consumer_newNDMethodsArray
 0002:00000598      ___somC_EventComm_Consumer_ClassInfo
 0002:000005A0      _EventComm_SupplierClassData
 0002:000005B0      _EventComm_SupplierCClassData
 0002:00000678      _EventComm_Supplier_try_pull_mp_tdcs00b58ce0
 0002:000006AC      ___somC_EventComm_Supplier_newNDMethodsArray
 0002:00000850      ___somC_EventComm_Supplier_ClassInfo
 0002:00000858      _has_event
 0002:0000085C      _event_data
 0002:00000A04      d3_1
 0002:00000A08      _EventChannelAdmin_ConsumerAdminClassData
 0002:00000A14      _EventChannelAdmin_ConsumerAdminCClassData
 0002:00000AB8      ___somC_EventChannelAdmin_ConsumerAdmin_newNDMethodsArray
 0002:00000C24      ___somC_EventChannelAdmin_ConsumerAdmin_ClassInfo
 0002:00000C2C      _EventChannelAdmin_SupplierAdminClassData
 0002:00000C38      _EventChannelAdmin_SupplierAdminCClassData
 0002:00000CDC      ___somC_EventChannelAdmin_SupplierAdmin_newNDMethodsArray
 0002:00000E48      ___somC_EventChannelAdmin_SupplierAdmin_ClassInfo
 0002:00000E50      _EventChannelAdmin_EventChannelClassData
 0002:00000E60      _EventChannelAdmin_EventChannelCClassData
 0002:00000F24      ___somC_EventChannelAdmin_EventChannel_newNDMethodsArray
 0002:000010B8      ___somC_EventChannelAdmin_EventChannel_ClassInfo
 0002:00001414      __ectbl__ EventComm_EventConnection::EventComm_EventConnection()
 0002:0000141C      __ectbl__ EventComm_Supplier::EventComm_Supplier()
 0002:00001424      __ectbl__ EventComm_Consumer::EventComm_Consumer()
 0002:0000142C      __ectbl__ EventChannelAdmin_ConsumerAdmin::EventChannelAdmin_ConsumerAdmin()
 0002:00001434      __ectbl__ EventChannelAdmin_SupplierAdmin::EventChannelAdmin_SupplierAdmin()
 0002:0000143C      __ectbl__ SOMObject::SOMObject()
 0002:00001444      d4_1
 0002:00001448      _CellClassData
 0002:0000145C      _CellCClassData
 0002:00001530      ___somC_Cell_newNDMethodsArray
 0002:000016EC      ___somC_Cell_ClassInfo
 0002:000017E4      d5_1
 0002:00001810      d79_1
 0002:00001810      ___CPPexceptionList
 0002:00001814      ___exceptFlags
 0002:00001818      ___throwFileName
 0002:0000181C      ___throwLineNumber
 0002:00001820      ___throwExceptionName
 0002:00001824      ___exceptStaticBuffP
 0002:00001828      ___exceptMemAllocVars
 0002:0000182C      ___ExceptStaticXbuff
 0002:000018AC      __ExceptVarsSize
 0002:000018C0      d83_0
 0002:000018C0      ___xxPersonality
 0002:000018C4      __fileinfo
 0002:000018C4      d87_0
 0002:000018C8      d95_0
 0002:000018C8      __turboFloat
 0002:000018CC      __argv_expand_ptr
 0002:000018CC      d103_0
 0002:000018D0      __wargv_expand_ptr
 0002:000018D0      d105_0
 0002:000018D4      d119_1
 0002:000018FC      __indStub:82
 0002:00001900      __indStub:83
 0002:00001904      __indStub:84
 0002:00001908      __indStub:86
 0002:0000190C      __indStub:87
 0002:00001910      __indStub:85
 0003:00000000      ___somC_EventComm_EventConnection_parentMtabs
 0003:00000000      b2_2
 0003:00000014      ___somC_EventComm_Consumer_parentMtabs
 0003:00000030      ___somC_EventComm_Supplier_parentMtabs
 0003:00000044      ___somC_EventChannelAdmin_ConsumerAdmin_parentMtabs
 0003:00000044      b3_2
 0003:00000054      ___somC_EventChannelAdmin_SupplierAdmin_parentMtabs
 0003:00000064      ___somC_EventChannelAdmin_EventChannel_parentMtabs
 0003:00000078      ___somC_Cell_parentMtabs
 0003:00000078      b4_2
 0003:00000094      b79_2
 0003:00000094      __DestructorCountPtr
 0003:0000009C      b117_0
 0003:0000009C      __pRawDllMain
 0003:000000A0      b119_2
 0004:00000000      ___xxInfo
 0004:00000000      t79_3
